:020000040000FA
:0400000024EF01F0F8
:10000800D8CF00F0E0CF01F0026EE9CF03F0EACFDD
:1000180004F0FACF05F0FBCF06F09DA816D09EA8F5
:1000280014D06750E96E020E6824EA6EEFCFADFF78
:100038007888672A000E6822676605D0020E686213
:1000480002D0676A686A6F4E9D98F2A815D0F2A22E
:1000580013D0F292F29878A48B947786E80ECF6E3C
:10006800900ECE6E9E90CD8077A806D0779877A216
:1000780003D00D0E7464742A9DAA67D09EAA65D019
:100088007786E80ECF6E900ECE6E9E90CD80ABA296
:1000980003D0AB98AB8859D0ABA415D0AE50E20EC4
:1000A800CF6EB40ECE6E9E90CD8077AC05D0779C87
:1000B800AC9A4A0EAF6E49D078A847D0AC9A7898D7
:1000C800778E779242D001EE80F06650E926AECF67
:1000D800EFFF77AC05D0779CAC9A4A0EAF6E2BD069
:1000E80078A829D06D50E96E020E6E24EA6EEFCF23
:1000F80079F001EE80F06650E926EF50791811E0AA
:10010800AC9A7898778C778E77927C0EAF6E9D98A4
:10011800AD6AAC8AE20ECF6EB40ECE6E9E90CD80E4
:100128000AD06D2A000E6E226D6605D0020E6E6230
:1001380002D06D6A6E6A5F0E716007D077BC05D019
:10014800662A600E666201D0666A9EA051D09E90B3
:1001580077A64AD07796F292F28878A48B8474C0F6
:100168007AF07A467A46F9507A44F926E80ECF6E44
:10017800900E36D0E90ECF6EBC0E32D0EA0ECF6E9E
:10018800E80E2ED0EC0ECF6E140E2AD0ED0ECF6EE8
:10019800400E26D0EE0ECF6E6C0E22D0EF0ECF6E34
:1001A800980E1ED0F00ECF6EC40E1AD0F10ECF6E80
:1001B800F00E16D0F30ECF6E1C0E12D0F40ECF6ECA
:1001C800480E0ED0F50ECF6E740E0AD0F60ECF6E16
:1001D800A00E06D0F70ECF6ECC0E02D0F80ECF6E62
:1001E800CE6ECD80778804D077A802D07798CD904E
:1001F8009EA218D09E92572E15D0050E576E2682B5
:10020800582E03D0020E586E2684592E0BD0140E89
:10021800596E26865A2E06D00A0E5A6E26885B2EEE
:1002280001D05B6E05C0FAFF06C0FBFF03C0E9FF03
:1002380004C0EAFF025001C0E0FF00C0D8FF100070
:1002480054EC0FF087EC0FF0D4EC0FF0000107EC42
:1002580010F00400D180F28CF28ECA8477B24FD0AD
:1002680077AE05D0779E6BC067F06CC068F06750BA
:10027800695C076E68506A58086E08AE02D0020EB4
:100288000826075008104DE06750E96E020E6824F2
:10029800EA6EEFAE2BD0096A020E0A6E67C00BF049
:1002A80068C00CF007C00DF00E6A0F6E4DEC08F038
:1002B8006F6E6F5036E0FF0A03E1C4EC0CF031D0EA
:1002C8006750E96E020E6824EA6EB20EEF6203D040
:1002D800070E746E01D0746A67C06BF068C06CF06A
:1002E80067C06DF068C06EF077821BD0C4EC0CF06C
:1002F8000706000E085A07500810C6E112D0ACA233
:1003080006D06F6604D0746A789877920AD077B866
:1003180008D077BC06D078A604D077B602D09D88DE
:10032800AC8A77B430D06550665C076E07AE02D0F1
:10033800600E072607C071F0075255E001EE80F005
:100348006550E926EFAE1AD0800E096E010E0A6ECE
:1003580065C00BF00C6A0BBE0C0607C00DF0600EF2
:100368000E6E0F6A4DEC08F0706E70503CE0FF0A9C
:1003780003E1B9EC0CF037D0778435D0B9EC0CF048
:10038800072EDCD730D001EE80F06550E926EF501B
:10039800830A0BE0330A0CE0010A14E0030A16E0B2
:1003A800060A18E05B0A19E01BD08EEC0CF01AD094
:1003B800000EE4EC0AF00FC008F010C009F06BEC76
:1003C80009F010D0010EE4EC0AF00CD0020EE4ECB7
:1003D8000AF008D00CEC0EF005D008EC0DF002D0B5
:1003E800B9EC0CF0779410EEA8F0076A080E0760D5
:1003F80051D0E650E6BE4CD0EA6A470E0724E96EB3
:10040800EF5046E024EE00F0200E0702F350D92604
:100418000C6A010E086E085232E0EA6A470E072499
:10042800E96E0850EF1425E0EA6A470E0724E96EE2
:10043800081CEF16DECF0BF0DDCF09F00F0E091404
:100448000A6E0938070B096E095006E0010A04E034
:10045800030A02E0010A0DE109C00DF00AC00EF01E
:100468000BC00FF00CC010F007C011F008507AEC68
:1004780007F0040ED9260C2AD8900836CCD707C026
:1004880024F0EA6A2F0E0724E96EEF50C3EC0EF051
:10049800072AACD726A274D02692040026AE05D02F
:1004A8005D2E03D0269E000EEBDB81B008D078A627
:1004B8000DD0722A140E726209D0789607D0726A2B
:1004C80078B604D0736602D0010E736E73520EE0D4
:1004D800732A330E73620AD0736AF29E9D98F29261
:1004E800F288AB889E9A9D8AF28E788610EEA8F0E4
:1004F800076A080E076044D0E650E6AE3FD0EA6AC5
:10050800370E0724E96EEFCF09F00750AFEC0EF075
:100518000A6EEA6A2F0E0724E96E0AC0EFFFEA6A3C
:100528004F0E0724E96EEFCF0CF0EA6A470E072456
:10053800E96EEFCF0DF00A5009180B6E010E086E28
:10054800085216E008500D1410E10C500B14081452
:100558000CE0EA6A370E0724E96E0850EF1AEA6AD7
:10056800470E0724E96E0850EF12D8900836E8D7EE
:10057800EA6A4F0E0724E96E0BC0EFFF072AB9D7C6
:1005880026A4F1D22694096A080E0960D1D0EA6A35
:10059800900E0924E96EEF50D8B4C8D024EE01F0CB
:1005A800200E0902F350D9260C90076A010E0A6E34
:1005B8000A52D8B4B0D0EA6A900E0924E96E0A50FB
:1005C800EF14D8B4A2D0DFCF0BF00B38070B086EAE
:1005D80001EE00F0080E0902F3500724D890E83421
:1005E800E926EE06000EEE5A01EE00F0080E0902AA
:1005F800F3500724D890E834E926EE50EE10D8A43A
:1006080084D0E26AD8900934A90FE16EE7BE57D0CA
:10061800E7AA16D0040ED9260B38F00B0B6E0F0E76
:10062800DF140B26040ED95E08C00DF00BC00EF0C7
:1006380007C00FF009C010F00A50C5DB0C8065D068
:100648000850020A03E0030E086215D0EA6A900E09
:100658000924E96E0A1CEF1608C00DF00F0E0B14E2
:100668000E6E0F6A07C010F009C011F00A507AEC3C
:1006780007F00C804AD0085202E0082C46D0EA6AFB
:10068800900E0924E96E0A1CEF16DD50DEBC08D076
:10069800EA6A2F0E0924E96E0A1CEF160C8035D081
:1006A800EA6A370E0924E96E0A50EF142EE1EA6A65
:1006B8002F0E0924E96E0A1CEF160C8026D0EA6A70
:1006C800900E0924E96E0A1CEF16EA6A270E09241F
:1006D800E96E0A50EF12EA6AA00E0924E96E0A5080
:1006E800EF140DE0EA6AA00E0924E96E0A1CEF1661
:1006F800EA6A980E0924E96E0A50EF1206D0EA6AEF
:10070800470E0924E96E0A50EF12040ED926072A6B
:10071800D8900A364DD70CA009D009C024F0EA6A4F
:100728002F0E0924E96EEF50C3EC0EF0092A2CD7DE
:1007380010EEA8F00D6A080E0D6055D1D8900D3452
:100748000F6EE6CF07F0E6CF08F008AE4AD1675043
:10075800695C096E68506A580A6E0AAE02D0020EC9
:100768000A26EA6A470E0D24E96EEF50D8B439D14B
:100778000ABE06D0C00E095C010E0A58D8B031D1A5
:1007880024EE00F0200E0D02F350D926040ED95E97
:10079800000EDA5A1068010E0E6E0E52D8B421D12E
:1007A800040ED926000EDA22102AEA6A470E0D2412
:1007B800E96E0E50EF14D8B411D1EA6A470E0D2431
:1007C800E96E0E1CEF16DECF0BF0DDCF0CF01290A9
:1007D800EA6A370E0D24E96E0E50EF14D8A4128081
:1007E800089612B008860B38030B28E178B0F6D0CB
:1007F800089812B00888EA6A270E0D24E96E0E5090
:10080800EF147BE0EA6A270E0D24E96E0E1CEF1642
:100818000896EA6A3F0E0D24E96E0E50EF14088818
:10082800D8B408980BC013F01980199207C014F0B7
:1008380008C015F01050C4EC08F0D0D00C38070BE5
:100848005CE178B05AD0EA6A270E0D24E96E0E50A2
:10085800EF1416E0EA6A270E0D24E96E0E1CEF1657
:10086800EA6A800E0D24E96E0E50EF14D880D8B4D1
:10087800D89003E212B0B2D040D012B03ED0AED081
:10088800EA6A900E0D24E96E0E50EF1420E1EA6A30
:10089800800E0D24E96E0E1CEF1612A00FD00E501C
:1008A800EF12030E0B14030A28E00CC013F010C05B
:1008B80014F00DC015F00E50B7DB90D00CC013F03B
:1008C80010C014F00DC015F00E50AEDB87D0EA6AE8
:1008D800800E0D24E96E0E50EF14D880D8B4D8904D
:1008E80003E212B003D009D012B007D0EA6A900E22
:1008F8000D24E96E0E1CEF1671D0030E0B14010ABD
:1009080007E0030A08E0010A08E0030A4DE005D001
:1009180012B003D049D012B047D00B38030B3AE1DC
:10092800EA6A900E0D24E96E0E50EF1457E1EA6A58
:100938003F0E0D24E96EEFCF11F008AC03D00E5036
:10094800111A07D010A003D00E50111202D00E1C9D
:1009580011160E5011140888D8B40898EA6A3F0E88
:100968000D24E96E11C0EFFF0C38070B020A09E1EC
:100978000CC013F010C014F00DC015F00E5054DB6D
:1009880008D0200E136E10C014F00DC015F00E50D4
:100998004BDB08860BC013F01980199207C014F0BE
:1009A80008C015F01050ECDBD8900B32D8900B3201
:1009B800030E0B14010A07E0030A08E0010A08E025
:1009C800030A0CE005D012B003D008D012B006D04C
:1009D800EA6A980E0D24E96E0E50EF12D8900E3682
:1009E800DCD60D2AA8D60E6A080E0E60ACD0675069
:1009F800695C096E68506A580A6E0AAE02D0020E27
:100A08000A26EA6A980E0E24E96EEF50D8B499D0F7
:100A18000ABE06D0E00E095C010E0A58D8B091D083
:100A2800E26AD8900E34A90FE16E24EE00F0200E91
:100A38000E02F350D926040ED95E000EDA5A116858
:100A4800010E0F6E0F527DE0040ED926000EDA2239
:100A5800112AEA6A470E0E24E96E0F50EF146EE170
:100A6800EA6A980E0E24E96E0F50EF1467E0E7AEBD
:100A780007D0EA6A900E0E24E96E0F50EF145EE17B
:100A8800EA6A980E0E24E96E0F1CEF16DECF0BF003
:100A9800DECF0DF0DECF07F0DECF08F0040ED95E12
:100AA800000EDA5A08C00CF00898EA6A370E0E24CD
:100AB800E96E0F50EF14D8A408880C38030B34E102
:100AC800EA6A3F0E0E24E96E0F50EF14088AD8B474
:100AD800089AEA6A270E0E24E96E0F50EF1408E010
:100AE800EA6A270E0E24E96E0F1CEF1608981CD030
:100AF8000D38070B020A09E10DC013F011C014F0FC
:100B08000EC015F00F5090DA08D0200E136E11C0E9
:100B180014F00EC015F00F5087DA0888EA6AA00EA4
:100B28000E24E96E0F50EF120CC013F019801982D1
:100B380007C014F008C015F0115022DBD8900F360A
:100B480081D70E2A51D778A00ED0076A080E076001
:100B580007D0EA6A470E0724E96EEF10072AF6D78E
:100B6800FF0AD8A4789026A659D026965E520DE0A2
:100B78005E060F0E5E1409E15E3A5E060F0E5E1405
:100B880003E0140E7DD85E8A5E3A5F5206E05F2E5F
:100B980004D0640E75D80A0E5F6E78A223D075064D
:100BA8000F0E75141FE1753A0F0E7514076E080EB7
:100BB800076014D0010E086E075005E0096ED89042
:100BC8000836092EFCD70850601406E0EA6A470E7A
:100BD8000724E96EEE687880752A01D07892753A14
:100BE8000A0E751282B219D05C2A78B407D00A0EA0
:100BF8005C620BD07884010E5F6E07D0020E5C62D7
:100C080004D078945F6A650E5C6E640E5C6203D0F3
:100C1800D19000EF00F0000101D05C6A26A832EF05
:100C280001F0269826AA32EF01F05B04076E080E41
:100C3800076032EF01F0E26AD8900734A90FE16E3D
:100C4800E7AE0FD007506124196E000E62201A6EAD
:100C5800EA6A3F0E0724E96EEF50F9EC0EF032EF26
:100C680001F007506124196E000E62201A6EEA6ABC
:100C7800370E0724E96EEF50F9EC0EF032EF01F071
:100C8800246E245205E024C05DF0268E8B9001D09E
:100C98008B8012001C6E010EEA6E1BC0E9FF1C4619
:100CA8001C461C44060FF924D8B0FA2AF96EEF6ADC
:100CB800000E00003BD0140EEF6E000E37D01E0E53
:100CC800EF6E000E33D0280EEF6E000E2FD0320ECE
:100CD800EF6E000E2BD03C0EEF6E000E27D0500E9C
:100CE800EF6E000E23D0640EEF6E000E1FD07D0E47
:100CF800EF6E000E1BD0960EEF6E000E17D0C80ECA
:100D0800EF6E000E13D02C0EEF6E010E0FD0900E6A
:100D1800EF6E010E0BD0F40EEF6E010E07D0580ED9
:100D2800EF6E020E03D0200EEF6E030EEC6E120073
:100D3800186E010EEA6E17C0E9FF18461846F950FA
:100D48001844F926E80EEF6E030E3BD0DC0EEF6E6A
:100D5800050E37D0D00EEF6E070E33D0B80EEF6EFB
:100D68000B0E2FD0A00EEF6E0F0E2BD0880EEF6E4D
:100D7800130E27D0700EEF6E170E23D0280EEF6ECD
:100D8800230E1FD0E00EEF6E2E0E1BD0500EEF6E0E
:100D9800460E17D0C00EEF6E5D0E13D0300EEF6EFC
:100DA800750E0FD0A00EEF6E8C0E0BD0100EEF6EDE
:100DB800A40E07D0800EEF6EBB0E03D0600EEF6E50
:100DC800EA0EEC6E1200116EEA6A2F0E1024E96E1C
:100DD800EFCF13F00F5005E0166ED8901332162E91
:100DE800FCD7030E13160E14136214D026900EB4FB
:100DF80026802F0E1024246E1150DEEC0EF0269063
:100E08000EB626802F0E1024246ED8901134DEECF6
:100E18000EF013D026900EB026802F0E1024246ECC
:100E28001150DEEC0EF026900EB226802F0E102404
:100E3800246ED8901134DEEC0EF010C024F0EA6A6B
:100E48002F0E1024E96EEF50C3EC0EF00E380F0B86
:100E58000E6E080E1002F3500F24126EEA6A900EFE
:100E68001024E96E111CEF160D50020A03E0010A66
:100E780019E02FD0D89012341B6E0E500BDF01EE04
:100E880000F0D8901234E926EECF14F0EECF15F02A
:100E9800145015101EE0EA6A900E1024E96E1150E5
:100EA800EF1217D0D8901234176E0E5041DF01EEB2
:100EB80000F0D8901234E926EECF14F0EECF15F0FA
:100EC8001450151006E0EA6A900E1024E96E1150CD
:100ED800EF12D8901532143201EE00F0D890123487
:100EE800E92614C0EEFF15C0EEFF1200126E0D5277
:100EF80002E00D2C0AD00FBC08D0EA6A900E11242B
:100F0800E96E1250EF14D8A41200EA6A370E1124C1
:100F1800E96E1250EF146AE0080E1102F350102423
:100F2800136E0D5203E0020E0D6206D0D8901334F2
:100F38001B6E0E50AFDE0AD00D4C03D0030E0D62AF
:100F480005D0D8901334176E0E50F2DE01EE00F083
:100F5800D8901334E926EECF15F0EECF16F00D50E9
:100F6800020A07E0010A0FE0030A30E0010A2EE056
:100F78005AD01550161007E1EA6A2F0E1124E96EAF
:100F88001250EF1250D0EA6A900E1124E96E1250F6
:100F9800EF1449E1EA6A2F0E1124E96E1250EF1A94
:100FA800D8901632153201EE00F0D8901334E926A5
:100FB80015C0EEFF16C0EEFF1550161034E0EA6AB1
:100FC800900E1124E96E1250EF122DD0EA6A2F0EFE
:100FD8001124E96E1250EF121550161024E0EA6A37
:100FE800900E1124E96E1250EF121DD00D50020A16
:100FF80007E0010A05E0030A09E0010A07E013D047
:10100800EA6A900E1124E96E121CEF16EA6A900E35
:101018001124E96E1250EF1406E1EA6A2F0E11242A
:10102800E96E121CEF161200166E0F0E1314176ECF
:101038001338070B186E020A02E0186629D0080E4A
:101048001502F3501424196E175206E0D89019347B
:101058001B6E17501FDE16D0020E186209D001EE63
:1010680000F0D8901934E926140EEE6EEE6A0AD014
:10107800186608D001EE00F0D8901934E926010E60
:10108800EE6EEE6AEA6A900E1524E96E1650EF12BB
:1010980012000B500924E96E0C500A20EA6EEFCFBB
:1010A80011F011AC26D011AA21D00D4C1ED00BC0C6
:1010B80012F00CC013F0122A000E132212500E6206
:1010C80005D013500F6202D0126A136A1250092415
:1010D800E96E13500A20EA6EEFCF10F0030E106489
:1010E80003D0100E10640CD0FF0C000C060E106E0E
:1010F80007D011AA03D0040E106E02D0020E106E93
:10110800116A0B500924E96E0C500A20EA6EEF5060
:10111800111A0B2A000E0C220B500E6205D00C502F
:101128000F6202D00B6A0C6A1004126E125223E08E
:101138000D060DBE02D00D52D8B4000C0B50092478
:10114800E96E0C500A20EA6EEFBEFF0C0B50092422
:10115800E96E0C500A20EA6EEF50111A0B2A000EA5
:101168000C220B500E6205D00C500F6202D00B6A95
:101178000C6A1206DBD7113C02D010501200FF0C8B
:10118800166E1338030B176E19B23CD0199415BCA0
:1011980019841F0E1516175005E0010A10E0030AFE
:1011A80023E02FD019A405D016501426000E1522BE
:1011B8005ED0D89016301426000E152258D0158A05
:1011C800158819B405D016501426000E15224FD0D4
:1011D800D89016301426000E1522010E1616165039
:1011E8001588D8B4159843D0158AD8901630142687
:1011F800000E1522010E161616501588D8B415982B
:1012080036D0120078B012003F0E1516175005E0C0
:10121800010A0EE0030A1DE029D0159615B81586B7
:10122800159815BA1588100E13BC151A159A1FD0E3
:10123800159615B81586080E13BC151A158819B019
:1012480006D0159A158615A812D0159610D0158AAD
:101258000ED0D88015AED890153214321598D8B063
:101268001588158A080E13BC151A01D01200D890DB
:1012780014361536D8901432186A6950E96E020E81
:101288006A24EA6EB00E1710EE6E18508ADB186EDC
:101298006950E96E020E6A24EA6E14C0EFFF185016
:1012A80080DB186E6950E96E020E6A24EA6E15C07A
:1012B800EFFF185076DB186E6950E96E020E6A244B
:1012C800EA6E181CEF6E000E6CDB140ED9D40850B1
:1012D8000914FF0AD8B4120010EEA8F00D6A080E1F
:1012E8000D6038D0E6CF0AF0E6CF0BF00BAE30D069
:1012F8000BAC2ED0070E0B1624EE00F0200E0D02BC
:10130800F350D926106A010E0E6E0E5221E0DFCF7F
:101318000CF00C38030B13E108500A6210D0095086
:101328000B620DD001EE80F06550E9262690EFBAE9
:1013380026803F0E0D24246E0E50DEEC0EF0040EB7
:10134800D926102A0A2A000E0B22D8900E36DDD78D
:101358000D2AC5D712001C6ED9CF21F0DACF22F0A2
:1013680024EE00F0200E1B02F350D926040E1A02B8
:10137800F350D926DECF1EF023B02CD01E38030B35
:101388001962F1D0195014E123A2EDD0269023B4AC
:101398002680370E1B24246E1C50DEEC0EF0EA6A01
:1013A800470E1B24E96E1C50EF12140E69DCDBD0CB
:1013B800269023B22680370E1B24246E1C50DEECA8
:1013C8000EF0EA6A470E1B24E96E1C50EF12140E49
:1013D80057DCC9D01966C7D023A2C5D01AB007D028
:1013E800EA6A900E1B24E96E1C1CEF1608D0EA6A04
:1013F800900E1B24E96ED8901C30FF0AEF161AB025
:1014080027D0268023B42690370E1B24246E1C5028
:10141800DEEC0EF0268023B426902F0E1B24246EBB
:101428001C50DEEC0EF0269023B42680370E1B24C9
:10143800246ED8901C34DEEC0EF0269023B426805F
:101448002F0E1B24246ED8901C34DEEC0EF07FD0B7
:1014580023B41FD02690370E1B24246E1C50DEECBC
:101468000EF026902F0E1B24246E1C50DEEC0EF07E
:101478002690370E1B24246ED8901C30DEEC0EF01C
:1014880026902F0E1B24246ED8901C30DEEC0EF014
:101498005ED0DFCF1FF01F5006E0050A04E00F0AF8
:1014A80002E0050A27E126901FB22680370E1B248A
:1014B800246E1C50DEEC0EF026901FB226802F0EF4
:1014C8001B24246E1C50DEEC0EF026901FB02680E4
:1014D800370E1B24246ED8901C30DEEC0EF02690BC
:1014E8001FB026802F0E1B24246ED8901C30DEECF3
:1014F8000EF02DD02680370E1B24246E1C50DEECF7
:101508000EF02680370E1B24246ED8901C30DEEC9B
:101518000EF0040ED95E5F0EDF1417E0060E1A14E3
:10152800206E080E1B02F35020241D6E01EE00F001
:10153800D8901D34E926010EEE6EEE6AEA6A900E26
:101548001B24E96ED8901C30EF12040ED9261BC05C
:1015580024F0EA6A2F0E1B24E96EEF50C3EC0EF05C
:10156800140E44EC06F0DE50DCBE25D0D8901E32B6
:10157800D8901E32030E1E14010A05E0030A0CE07F
:10158800010A13E018D023A216D0EA6A980E1B2489
:10159800E96E1C50EF120FD023B20DD0EA6A980EF4
:1015A8001B24E96E1C50EF1206D0EA6A980E1B2421
:1015B800E96E1C50EF1221C0D9FF22C0DAFF1200D9
:1015C800086ED3D901EE80F06550E926D890EF3443
:1015D8000F6ECBD901EE80F06550E9260F0EEF149F
:1015E800106ED89010320F3201EE80F06550E92667
:1015F8001590EFBC15800850020A05E0030A08E0C0
:10160800010A19E02DD015B02ED00F681068FF0C14
:1016180015B029D0EFBA02D0EFA804D0EFAA05D0B0
:10162800EFA803D00F681068FF0CEFAA02D0EFA84C
:10163800EF88EF8C18D015A003D00F681068FF0C46
:10164800F80E0F5C030E10580EE3FC0E0F5C030E31
:10165800105809E20FC016F010C017F062D903D075
:101668000F681068FF0C10EEA8F0096A080E0960F0
:101678004FD1E6CF11F0E6CF12F012BE47D124EEDB
:1016880000F0200E0902F350D926DD50159612BA43
:101698001586070E12160E6A0850010A06E0010A9E
:1016A80004E0020AD8B492D031D1010E0D6E0D5269
:1016B800D8B42CD10F50116221D0105012621ED014
:1016C80001EE80F06550E9261592EFB8158201EE1B
:1016D80080F0E9261594EFBA158408C019F0239014
:1016E80015B62380239215B22382239415B423843C
:1016F8000EC01AF009C01BF00D502DDEDCCF0BF028
:10170800030ED926000EDA22DFAE59D0300EDF14D0
:101718000C6E0C38086253D0070EDD14146EDECF41
:1017280013F00F5013624BD01050146248D001EEE2
:1017380080F06550E9261592EFB8158201EE80F029
:10174800E9261594EFBA1584086604D0040EDFBCA8
:10175800151A03D0020EDFBC151AD8900B32D89098
:101768000B32030E0B14010A05E0030A06E0010A16
:1017780006E025D015B203D022D015B220D0D890DB
:101788000B32D8900B32030E0B160B5007E0010AF0
:1017980002E0030A14E1159215B415820BC019F082
:1017A800239015B62380239215B22382239415B46F
:1017B80023840EC01AF009C01BF00D50CCDD0E2A90
:1017C800112A000E1222D8900D3671D7010E0D6E17
:1017D8000D52D8B49BD00F50116229D0105012620C
:1017E80026D001EE80F06550E926EFAA03D00E2A34
:1017F800D8900D3601EE80F06550E9261592EFB8C5
:10180800158208C019F02390239215B223822394DD
:101818000EC01AF009C01BF00D509DDD01EE80F0DE
:101828006550E926EFAA03D00E06D8900D32159818
:10183800DCCF0BF0030ED926000EDA22DFAE5CD027
:10184800300EDF140C6E0C38086256D00F0EDD1403
:10185800146EDECF13F0D890143213320F50136287
:101868004BD01050146248D0DD5001EE80F0655026
:10187800E926EFBA03D0DEA003D03ED0DEA03CD0EC
:1018880001EE80F06550E9261592EFB81582020E38
:10189800DFBC151AD8900B32D8900B32030E0B14FC
:1018A800010A05E0030A06E0010A06E025D015B2A0
:1018B80003D022D015B220D0D8900B32D8900B325A
:1018C800030E0B160B5005E0010A07E0030A05E0BA
:1018D80013D0159415B2158415820BC019F02390F6
:1018E800239215B22382239415B423840EC01AF0D0
:1018F80009C01BF00D502FDD0E2AD8900D36157833
:1019080015B896D7112A000E122262D7092AAED628
:101918000F5012002AD8BAA503D078820A0E756E25
:101928001200BAA721D001EE80F06550E926EFB881
:101938001BD0030E1614196ED890193601EE80F0DC
:101948006550E926EFBA1980080E19600DD0E26AD1
:10195800D8901934A90FE16EE7AE06D0EA6A470EAF
:101968001924E96EEE687880120001EE80F0655067
:10197800E926EF6A652A600E656201D0656A120081
:101988006750E96E020E6824EA6EEF6A672A000E55
:101998006822676605D0020E686202D0676A686AC4
:1019A80012001A6E6950E96E020E6A24EA6EEF5050
:1019B8001A1A692A000E6A22696605D0020E6A623E
:1019C80002D0696A6A6A1A501200A80E126E136A67
:1019D800146AB80E156E45DA116A106A040E1060A2
:1019E8000ED0136E1150126E400E1124146EB80EE4
:1019F800156A152236DA400E1126102AEFD7D0DAEA
:101A0800268C01DB269C1200B0DFBAA31200ADDFE2
:101A180001EE80F06550E9267C0EEF626FD0A5DFFD
:101A280001EE80F06550E926EFCF0CF09EDF9DDFD8
:101A380001EE80F06550E926EFCF09F096DF01EE60
:101A480080F06550E926D890EF34086ED88009AE4A
:101A5800D890093208323F0EB8150B6EB9C00AF09B
:101A680078B406D008500A6249D009500B6246D0B3
:101A78007CDF7BDFFC0E0C14200A0BE0080A09E06F
:101A8800040A15E04C0A21E0080A1FE00C0A2AE0C3
:101A980035D078A409D0BAAF07D00CC00DF008C073
:101AA8000EF009C00FF02BD8010E89D827D078B4D2
:101AB80007D00CC00DF008C00EF009C00FF01FD8F9
:101AC800BAAF1CD07F0E7BD819D078A406D0D1D855
:101AD800BAAF14D0400E73D811D0BAAF0FD0000EE1
:101AE8006ED80CD078B406D0C4D8BAAF07D0400EA0
:101AF80066D804D0BAAF02D0000E61D8120015EE35
:101B080000F0E70EE66E0E0EE66E7C0EE66E0DC079
:101B1800E6FF100EE66ED8900E360F36D8900E32CD
:101B28000FC0E6FF0EC0E6FFE66A166A01EE80F017
:101B38006550E926EFCF14F014C018F018380F0BD1
:101B4800186E13DF01EE80F06550E926EFCF15F02F
:101B580015C017F0179E14B0178E18500FE1160E07
:101B680017600CD0A80E1724E96E000E1820EA6E34
:101B7800EFCF16F0140E44EC06F013D0160E175CD7
:101B8800010E18580EE2160E175E000E185A17505E
:101B9800E96E040E1824EA6EEFCF16F0140E44EC2A
:101BA80006F0149216BE148214C0E6FF15C0E6FFB4
:101BB8007F0E1614E66EE66AE66A788A12000D6EE3
:101BC8000E6A6950E96E020E6A24EA6EB40EEE6E71
:101BD8000E50E7DE0E6E6950E96E020E6A24EA6E58
:101BE8006F0EEF6E0E50DDDE0E6E6950E96E020E5E
:101BF8006A24EA6E0DC0EFFF0E50D3DE0E6E6950F8
:101C0800E96E020E6A24EA6E0E1CEF6E000EC9D64B
:101C1800096AABDE01EE80F06550E9266F0EEF62CF
:101C280027D078AA25D0789A15EE00F06950E96E89
:101C3800020E6A24EA6EE6CFEFFF0950B2DE096EA3
:101C4800020EE75C086E6950E96E020E6A24EA6EBD
:101C5800E6CFEFFF0950A5DE096E082EF4D76950CC
:101C6800E96E020E6A24EA6E091CEF6E000E99D620
:101C7800120001EE80F06550E926EFCF0FF075DE17
:101C880001EE80F06550E926EFCF0EF00E9E0FB002
:101C98000E8E6BDE01EE80F06550E926EFCF0DF079
:101CA8000D9E0FB20D8E0F380F0B0F6E140E0E62B5
:101CB80002D00F5205E0150E0E620BD00F6609D048
:101CC800AA0E0D6201D081DEA10E5E6E140E44EFE5
:101CD80006F00F5013E1140E0E6010D0A80E0E245B
:101CE800E96E000E0F20EA6E0DC0EFFF04000EC073
:101CF80019F00FC01AF00D5078D81BD0160E0E5CD4
:101D0800010E0F5815E2160E0E5E000E0F5A0E50F9
:101D1800E96E040E0F24EA6E0DC0EFFF0400400EBA
:101D28000E24196E000E0F201A6E0D505ED801D0C9
:101D3800120036D90F500AE1100E0E6007D0010EBE
:101D48000E14010A03E1268C5ED9269C510E5E6EA4
:101D5800140E44EF06F0196EF00E80161950802606
:101D6800899881CF1AF01A9082BA1A808988EA6A0B
:101D7800880E1924E96EEF501A1A1A501200256EAF
:101D8800EA6A880E2424E96EEF50251A010E93168C
:101D9800949A25C081FF25A0829A25B0828AF00EE8
:101DA8008016080E2424802689988988FE0E9312AE
:101DB800948A1200256E24C0E9FFEA6AD890EF14CD
:101DC800D8A4D88026A003D02550EF1202D0251C15
:101DD800EF161200A6B2FED71CC0A9FF1DC0AAFFAD
:101DE800A69EA69CA680A85012001B6E19C01CF0C7
:101DF8001AC01DF0EFDF1B1832E0A6B2FED71BC0D9
:101E0800A8FF19C0A9FF1AC0AAFFA69EA69CA6846F
:101E1800F29E550EA76EAA0EA76EA682F28EA69403
:101E2800632A000E6422E90E635C030E64580EE315
:101E3800636A646A612A000E6222F10E615C030E15
:101E4800625804E3400E616E010E626E19C01CF008
:101E58001AC01DF0BFDF1B1802E0D8901200D8800E
:101E68001200A68EA69CF86A1550F76EC00E1414C0
:101E7800F66E12C0E9FF13C0EAFF400E166E0900A5
:101E8800F552F5CFEEFF162EFAD712000AC0F6FF6C
:101E98000BC0F7FFF86AA68EA69C0800F550120042
:101EA8000F0EC16E070EB46E300E806EC00E926EAD
:101EB800816A9368D50E826EEA0E946ED0A60AD017
:101EC800D0A408D000EE00F00F0EEE6AEA62FDD74B
:101ED800E9AEFBD7F19CF298F2924A0EAF6EAC8451
:101EE800AC98AB8E9D989D9AAB98D56A800ECD6EB6
:101EF8009E909D80490ECA6ECC6A7C0ECB6E9E92D7
:101F08009D82B16A1200572A582A592A592A5A2AF0
:101F18005B2A140E0A6EB80E0B6EB8DF096E140E2B
:101F28001C6E1D6A57DF091809E009C0A8FFA684BE
:101F3800550EA76EAA0EA76EA682A69400EEA8F06C
:101F4800076A086AA68407C01CF008C01DF042DFB3
:101F5800EE6E550EA76EAA0EA76EA682072A000E71
:101F68000822085003E1150E0764EDD704EE00F0CF
:101F7800400E076E086A07C01CF008C01DF02ADF73
:101F8800EE6E550EA76EAA0EA76EA682072A000E41
:101F98000822400E075C010E0858EDE3A6941200D3
:101FA8006068010E126E10EEA8F0136A080E136036
:101FB80029D0EA6A880E1324E96EEF6A010E156EBD
:101FC80024EE00F0200E1302F350D926E650E6BEA8
:101FD80003D0D92A121C6016176A200E17600ED07B
:101FE800DFAE06D0EA6A880E1324E96E1550EF12A8
:101FF800D8901536040ED9261726EFD7D890123662
:10200800132AD4D71200010E9316949A60C081FF48
:1020180060A0829A60B0828A899A898AFE0E931299
:10202800948A8B981C6E030E1D6ED4DE616E1C683C
:10203800030E1D6ECFDE626E1890F10E615C030E0A
:10204800625805E31880400E616E010E626E269A92
:10205800BAB1268A26AA15D026AC05D061C016F0DA
:1020680062C017F005D06128166E000E6220176E48
:10207800F10E165C030E175804E3400E166E010E9F
:10208800176E070E126E12BE72D0E26AD890123422
:10209800A90FE16E26AA5ED018A002D0136A0AD052
:1020A800125061241C6E000E12BEFF0E62201D6EBF
:1020B80091DE136E040012501624196E000E12BE23
:1020C800FF0E17201A6E135090DEE7BE3DD0EA6A65
:1020D800370E1224E96E13C0EFFFE7AA2FD0EA6A81
:1020E8002F0E1224E96E13C0EFFF12C024F0EA6A23
:1020F8002F0E1224E96EEF5042DE020E156E010E0D
:10210800146E080E146026D0030E1314030A0BE194
:10211800196A23802382238414C01AF012C01BF08A
:102128001550AFEC09F0D8901332D8901332D890EC
:102138001536D8901536020E1426E3D7EA6A470EEC
:102148001224E96EEE6806D0EA6A3F0E1224E96EA0
:1021580013C0EFFFE7AE09D01250FDDD136EEA6A37
:10216800370E1224E96E13C0EFFF12068CD716C083
:1021780061F017C062F00400FE0E196E030E1A6EAD
:10218800615033DE04001968030E1A6E62502DD6B2
:10B800000080088010801880208028803080388058
:06B81000E71007000457D9
:10B84000230000002300000023000000230000006C
:10B85000230000002300000023000000230000005C
:10B86000230000002300000023000000230000004C
:10B87000230000002300000023000000230000003C
:10B88000230000002300000023000000230000002C
:10B89000230000002300000023000000230000001C
:10B8A000230000002300000023000000230000000C
:10B8B00023000000230000002300000023000000FC
:10B8C00023000000230000002300000023000000EC
:10B8D00023000000230000002300000023000000DC
:10B8E00023000000230000002300000023000000CC
:10B8F00023000000230000002300000023000000BC
:10B9000023000000230000002300000023000000AB
:10B91000230000002300000023000000230000009B
:10B92000230000002300000023000000230000008B
:10B93000230000002300000023000000230000007B
:0200000400F00A
:100000000080088010801880208028803080388010
:06001000E7100700045791
:100040002300000023000000230000002300000024
:100050002300000023000000230000002300000014
:100060002300000023000000230000002300000004
:1000700023000000230000002300000023000000F4
:1000800023000000230000002300000023000000E4
:1000900023000000230000002300000023000000D4
:1000A00023000000230000002300000023000000C4
:1000B00023000000230000002300000023000000B4
:1000C00023000000230000002300000023000000A4
:1000D0002300000023000000230000002300000094
:1000E0002300000023000000230000002300000084
:1000F0002300000023000000230000002300000074
:100100002300000023000000230000002300000063
:100110002300000023000000230000002300000053
:100120002300000023000000230000002300000043
:100130002300000023000000230000002300000033
:020000040020DA
:080000000507000100010001E9
:020000040030CA
:08000000FF021F08FF8181FFD0
:00000001FF
